:1000000001308A003B2900004D39E135EF36653972
:10001000A016A0266F3A6F392010D6127310A821AF
:1000200029103218301BA025C1254C050D005E306B
:1000300084008313000803192A280230F800F7010E
:10004000F70B2028F80B1F289730F700F70B26280E
:10005000800B1D2808009030D8008316860183127B
:10006000580886000130D9000230DC00FA30DE008A
:100070001720DC0B362808005D08DD03003A031961
:10008000552859080139013C031D4928C030D806BC
:100090004B283030D8068316860183125808860014
:1000A0001430DE001720D90A3C28080083160513F7
:1000B000831205130830F8005D280000F8176E2839
:1000C000F813E00C03180517031C051378176E28A6
:1000D0007813F80B61286C28000005170130F70031
:1000E0008401840B7128F70B70280E308400840B78
:1000F00077280000F81B6028781B68280800DC01BE
:10010000831605168312051A97280130DD003C205E
:10011000DC0A5C08283C031D96288316860183129E
:1001200086014530E00056208A01002880280230F0
:10013000DD00FA30DE001720DD0B992883168601DA
:100140008312860108000408F800831685178312BD
:10015000851BA8280830F700DC01F717BF28F71324
:10016000BF280310851B0314DC0C7717BF287713F7
:10017000F70BB128780884005C08F800D428013017
:1001800084000030F71B5530F800F80BC528840BAD
:10019000C1280D30F71B0330F800F80BCD28F71BF2
:1001A000AF28771BB728B1288A11FC2983160317BB
:1001B0008C170C14000000000318052983120C088A
:1001C0007F390313DD0003170D080313DE00031747
:1001D0000F080313DF005D08E00056205E080317D8
:1001E0008D0003135F0803178F0083168C170C1400
:1001F0000000000083120313DC0BFF280229831682
:100200000317052924298316031783120C0D0E0DDD
:100210007F390313DD0003170D080313DE000317F6
:100220000F080313DF005D08E00056205E08031787
:100230008D0003135F0803178F008D0A03198F0ABF
:1002400003100313DC0BD6280800800803193A2991
:10025000DD010408DC005D10831B5D140008E00074
:1002600056205C08840083135D188317840A0319E1
:10027000850A25290800840183131F308305723005
:1002800083168F000F0805138312051783161F129C
:100290009F121B0880399B0007309C008312A0012D
:1002A000A1013330A2002E30A3003030A400A501FC
:1002B0002430A6004930A7006430A8003A30A900D5
:1002C0002030AA006930AB007230AC006D30AD0058
:1002D0007230AE006130AF006B30B0002E30B10034
:1002E0006330B2002030B3003130B4003530B50097
:1002F0003830B6003630B7002030B8003230B900A0
:100300003030BA003130BB003030BC002D30BD0081
:100310003030BE003830BF002D30C0003230C10058
:10032000C2002030C3003030C4003830C5003A303D
:10033000C6003330C7003530C8003A30C90033300A
:10034000CA00CB005A30CC002030CD006B30CE003C
:100350006130CF006B30D0006C30D1002030D20043
:100360002430D300D40183161F129F121B0880393A
:100370009B0083121F109412831606118614061216
:100380000130831294000030831694000108C739AD
:1003900008388100831290010030F800920000308C
:1003A00083169200061483129701073083169C006F
:1003B000050885000630F700F70BDC2900001C0853
:1003C00083120D1383169D0172308F000F08860172
:1003D0008312860107308316860083122B207F202C
:1003E00018121816851FFB29831605168312051A85
:1003F000FA297F20F229A3287808DA005A086D3CF0
:10040000031D3A2A2B20D90A1230DD003C2002308D
:10041000DC00C830DE001720DC0B092A4130E00088
:1004200056203230DE0017200630DD003C2002303E
:10043000DC00C830DE001720DC0B192A4230E00057
:1004400056203230DE0017200630DD003C2002301E
:10045000DC00C830DE001720DC0B292A4330E00026
:1004600056203230DE001720D90A7F204730E000C6
:100470005620F0295A08693C031D422A4930E00001
:100480005620F0295A08683C031D4A2A4830E000EB
:100490005620F0295A08663C031D522A4630E000D7
:1004A0005620F0295A08783C031D782A0430031797
:1004B0008D0000308F00031013300313DC00D620B2
:1004C00022308400831325210E3003178D00003065
:1004D0008F00031410300313DC00D6202630840074
:1004E000831325210D30E00056200A30E00056200D
:1004F0005A082F3C0318822A5A08403C031C822ABF
:100500003030DA025A080B3C031CF0292B20D90AA0
:100510000C30DD003C20DB015A085B020318952AF1
:100520000230DD003C20DB0A8C2A0230DC00C830BF
:10053000DE001720DC0B972A5330E00056203230C3
:10054000DE001720D90A7F204730E0005620F0292E
:02055000630046
:04400E00383FFC3FFC
:00000001FF
